:020000040800F2
:20000000200600204D0A00085101000851010008510100085101000851010008510100081F
:200020005101000851010008510100085101000851010008510100085101000851010008F0
:200040005101000851010008510100085101000851010008510100085101000851010008D0
:200060005101000851010008510100085101000851010008510100085101000851010008B0
:20008000510100085101000851010008510100085101000851010008510100085101000890
:2000A000510100084909000851010008510100085101000851010008510100085101000870
:2000C000510100085101000851010008510100085101000851010008510100085101000850
:2000E000510100085101000851010008510100085101000851010008510100085101000830
:2001000051010008510100085101000851010008510100085101000851010008510100080F
:200120005101000851010008510100085101000851010008510100085101000851010008EF
:20014000510100085101000851010008510100082DE9F04F684600F0D3BA2DE9F007B1E811
:20016000F807A0E8F807203AF9D1BDE8F00770472DE9F007CDB24FF001346C4323462546FF
:2001800026462746A046A146A246A0E8F807203AFBD1BDE8F007704770B506460C460025E9
:2001A000E30704D518222946304600F0BBFE0135102D4FEA5404F3D170BD00002DE9F04178
:2001C0004FF00056054612220D210F4800F0AAFEB0460D4C4FF400579620C4F8108000F013
:2001E00075FA9620276100F071FA022D07D19620266100F06BFA9620276100F067FA4FF48C
:20020000FA6000F063FAE5E700100140F7B5604B604D00934FF6FF7308220E212846ADF860
:20022000043000F07FFE08220F21284600F07AFE0A2000F047FA18220E212846AC6800F0B7
:2002400071FE18220F21284600F06CFE0A2000F039FAAA680220D2430023C4F38134C2F323
:200260008132C2F3400104F00205294303EB43030229DBB211D0032911D0012901D1013364
:20028000DBB2640052000128A4B292B203D1022B08D9022004E00120E3E70233F0E7012058
:2002A000FFF78CFF0C223C493C4D02FB03122A6048253B4C9268257300256573394D637207
:2002C0002D880432E58112F8045C0432002D3ED10C22012702FB03125268043212F8040C7F
:2002E0000432002843D10C2202FB0313DB786BB10222BDF8005000F18040114600F5843002
:2003000025F0040500F00EFEADF80050637A2648013B012B9EBFBDF8003023F48073ADF82A
:200320000030BDF80010FFF737FFBDF802101F48FFF732FFBDF804101648FFF72DFF1222CA
:200340000D21144803B0BDE8F04000F0EBBD12F8075C02AE06EB450512F8066C00FA06F728
:2003600035F8086C26EA070625F8086CABE712F8070C02AD05EB400012F8065C07FA05F638
:2003800030F8085C25EA060520F8085CA6E700BFFEE1270E001001403419000820060020EF
:2003A00004000020DC06002000080140000C014000280CBF4FF400524FF00052014B1A61A1
:2003C000704700BF0010014003460144104610B5064C8B4200D110BD13F8012B82EA10221B
:2003E00034F8122082EA002290B2F2E7A219000803688B4238BF1A700368013303607047C1
:020000040800F2
:200400002DE9F04F8046174687B01D464B1E02900093C118BA461AF8012B52B9029B8B42B0
:2004200000F2FA801A700298A0EB080007B0BDE8F08F252A04D002A8FFF7DAFF5746E9E7B5
:20044000002634461CE0A2F16303152B26D8DFE803F072562525253E562525252525491131
:2004600025255B2558252511392A21D9582A15D144F4807444F0100436E055F8046BBA46F4
:20048000574617F8012B782A08D8622ADBD8302A0BD0E9D8232A05D02A2AEED002A8FFF7F9
:2004A000A7FFB7E744F48064E9E744F40064E6E7A2F130063A4612F8013BA3F1300009281F
:2004C000DDD80A2000FB06361746303EF2E79AF80130682B06BF44F480540AF1020744F4FF
:2004E0000054CCE744F00804E30455F8049B04F4007224D55FFA89F924F4007432E044F4CE
:20050000007444F00A04EFE755F8044B2644A6EB040A14F8012B52B9BAF1000F7FF77AAF0E
:20052000202202A8FFF764FF0AF1FF3AF4E702A8FFF75EFFEBE755F8042BD2B2AEE7A0045F
:2005400037D59AB30FFA89F9B9F1000FD4DA230505D52D2202A8FFF74BFF24F40074013E4A
:20056000C9F1000960050FD504F01F0ABAF1080F02D0BAF1100F07D1302202A8FFF738FFF3
:20058000BAF1100F18D0013E0DF10C0AB9F1000F18D130230DF10D0B8DF80C3014F4006F13
:2005A00014BF30222022ABEB0A0327E01FFA89F9A2E7002AA0D0C7E7782202A8FFF718FF6D
:2005C000023EE1E7D346174A14F4807F164808BF104604F01F02B9FBF2FC02FB1C9E10F8A1
:2005E0000EE00BF801EBCE467245E146F3D9D5E702A80193FFF7FCFE019B013EB342F7DBD4
:20060000A30503D52D2202A8FFF7F2FED3453FF401AF1BF8012DF6E788459CBF009B08F89F
:20062000032000E7A51C0008941C00080CB407B504AB53F8042B0193FFF7E2FE03B05DF818
:2006400004EB02B070470000EFF3088181F30988022181F31488BFF36F8F104B83F308888E
:200660000F4B104A9A605A6942F404725A615A6A42F4E0225A624FF07F42DA614FF47F02EB
:200680001A62BFF34F8FBFF36F8F6FF07F42A3F54F635A6001221A60704700BF2002002025
:2006A00000ED00E000000008054A936891685B1A23F07F43984202D9C01A0B46F6E7704764
:2006C00010E000E000EBC000FFF7EEBF42F228335843FFF7E9BF000008B572B6054800F012
:2006E0007FFBBFF34F8FBFF36F8F034B034ADA60FEE700BFB61C000800ED00E00400FA051D
:20070000F7B50446EFF30382006AD2B2410704F1240341D5EFF309851E4605F120070F2AEA
:2007200040D82249DFF8A8C010F0080F204808BF6046AB6900901F4800F052FBEB681E480A
:200740000093D5E90123296800F04AFBE368216800931A48D4E9012300F042FBE3692169B1
:2007600000931748D4E9052300F03AFB236A296913F0040FAB6918BF3A46009308BF32460B
:200780006B69104800F02CFB3A463146EB690E4800F026FBFFF7A0FFEFF309871D4604F105
:2007A0004406BCE70949103ABCE700BFC81C0008D21C0008E11C0008051D0008351D0008E3
:2007C000651D0008951D0008C51D0008C41C0008D91C0008064B074A1B68926803F07F4035
:2007E0001043834238BF00F17F40C043704700BF2406002010E000E008B5FFF7EBFFC24305
:020000040800F2
:2008000003460448044940F8042B1944BDE8084000F04EB82406002020AA440010B500F042
:2008200081F8094B094C9B68094944F8043B2046002200F037F8FFF7CDFF06490144204663
:20084000BDE8104000F034B810E000E024060020F907000820AA44000C22114BB0F5803FA9
:200860001A600FDA0D284FF00702B8BF0D209A620C380122D8620A4B5A6100221A610D227B
:200880001A60704741F61F429A624FF4617290FBF2F04FF6FF723238904228BF1046E8E712
:2008A000002C01400123C0E90112C36070470000F8B504460D46EFF31186731EDBB23F2BC6
:2008C00002D9402383F31188E368154F012BF6B207D03A463B689C42D96814D101231160B5
:2008E000E3602560FFF776FF3B680246281A0C4D6BB9E3602C603B68A34201D1FFF7ACFF51
:2009000086F31188F8BD03F10C020B46E3E71968891A8142EDDA03F10C05DB68E8E700BF6F
:20092000380600200022064B5A600122DA604022044B83F819234FF000721A60704700BFC6
:20094000002C014000E100E00022F8B501270B4B0B4E1A61346804B9F8BD2568FFF73AFF7E
:20096000281A0C2803DDBDE8F840FFF775BFE368E7603360D4E901309847EBE7002C0140E9
:2009800038060020F8B532F01F0506460F4614460CD083070AD12A46FFF7EAFB04F01F0468
:2009A00072191444A24203D13046F8BD3246F8E702F8017BF6E7F8B532F01F0706460D4633
:2009C000144610D040EA01039B070CD13A46FFF7C4FB3D44F31904F01F04013B2C44A542C4
:2009E00003D13046F8BD3346F7E715F8012B03F8012FF4E703460246D01A12F8011B002998
:200A0000FAD1704708B5FFF7E5FE044B186000201871BDE80840FFF7CBBC00BF3C060020C3
:200A200008B5FFF7EFFF0122024B1A720022DA6008BD00BF3C06002008B5FFF7E3FF002220
:200A4000014B1A7208BD00BF3C060020B548B6492DE9F84F884203D0B44A121AFFF7ABFF18
:200A6000B348B44A0021121AFFF78CFF0022B24B19681A600522B14B9A614FF08062A3F5BE
:200A800088335A604FF6FF72C3F80C28AC4A03F500635A604FF044321A6000BF00BF9B6881
:200AA000A84A6FEA9333A84C03F001039142237408D03BB9A54BA64A1B681268591C01D0E1
:200AC0009D46904700F0CAF9FFF7A8FE00F096F900F0B2F9FFF79AFB9E4B9F481F789F4B17
:200AE000394693F80080DFF8A092424600F078F900F0C0FA9A4D00F017FFFFF76BFE94F8F8
:200B000008A0BAF1010F6AD0BAF1020FF3D1504600F0E0FE021E0FDBE168A66960690E44D7
:200B2000861B9642A8BF164650463246294400F0DDFEE2683244E260E668012E14DDA269B8
:200B400026F0010602F100623146284602F5005200F048FAA369E2683344921B2846A91919
:200B6000A361E260FFF727FFD4E905329A42C2D3032000F0B5FE0028BDD04FF6FF726169B3
:200B80007248FFF721FC774BB0F1000A764A514608BF1A46754800F023F9BAF1000318BF4F
:200BA000012301262B702672FFF72CFF32462946032000F0A1FE0023E360BAF1000F9AD073
:200BC0006669DFF888A106F1006606F50056564591D9504600F0F2F90AF5806AF7E72368D0
:200BE000C31A4B4506DD2060207980F001002071FFF7DEFB022000F06DFE061E0CDBE168EA
:020000040800F2
:200C0000C1F50063B34207D902203246294400F06DFEE0683044E060E368012B7FF66BAF82
:200C20006A789342FFF467AF032000F059FE00283FF461AF2E78012095F801A0FFF7B8FB81
:200C4000012E2CD00B2E56D0002E67D1BAF1030F64D1A978002961D110224548FFF792FEF1
:200C6000444B227C1F705A60434A83F8018003F1100153F8040B8B4242F8040BF9D12226EE
:200C800000236B70237A012B01D1FFF7BBFE32462946032000F030FE0023E3602BE7BAF1C1
:200CA000060F3BD1D5F802A01AF0030F18D1334B1A68334B03EB82239A451AD800F062F972
:200CC0000AF1006B214E0BF5005BB3450BD80223002651462B48C4E905A6237200F080F85F
:200CE0006E700226CEE7304600F068F906F58066EBE70D26F4E7BAF1030F0FD1AB7813F0EE
:200D0000FE0F0BD1012B07D100F0D2F94FF4FA70FFF7DCFCFFF7E0FC0226B1E701236B701F
:200D2000DFE700BF040000206C1F00082000002020060020AC0700200000002000100240AC
:200D400044444448EFBEADDE3C0600200020000804200008A1190008F11D0008A0190008F8
:200D6000AC070020EE1D0008E91D00082E1E0008BE07002004000020AE070020D80600204F
:200D800000E0FFFF1C1E000840771B0070B502460B46EFF3108404F0010472B60D25802139
:200DA0000D48FFF72DFB0C490C4A11F8013B13B904B962B670BD0A2B07D00D2BF5D016687B
:200DC000360607D55360F0E700BF16683606FBD55560F4E700BFF2E7580600200038014009
:200DE0000FB407B504A951F8040B0191FFF7CEFF03B05DF804EB04B07047000010B50B4A9E
:200E00000B4C9369204643F4804393610922114600F088F818220A21204600F083F81822C9
:200E2000044B9A6042F20C02DA6010BD001002400008014000380140064B5A68DA6842F085
:200E40002002DA600022044B83F8252320225A60704700BF0038014000E100E008B5FFF7A3
:200E6000F3FB2B4B2B4A1B889BB2102B136003D0202B45D0142300E0062353601222264B30
:200E80001A60A3F580531A6842F480321A601A68910337D5214A5A601A6842F080721A6022
:200EA0001A68920130D55A6842F002025A605A6802F00C02082A29D11A6822F001021A6067
:200EC0000722DA6140F61D029A6101225A614FF08062134B5A604FF0443302F1705202F5E5
:200EE000843253601360C2F80434C2F80034C2F80438C2F80038BFF34F8FBFF36F8F08BD49
:200F00000A23BAE700BFC2E700BFC9E700BFCEE7E0F7FF1FD80600200020024000C41D0082
:200F200000000140130914BF01234FF48033072903FA01F330B503614FF00F0402F00F02A8
:200F40000AD9083945688B009C4025EA040402FA03F32343436030BD036889008C4023EA8D
:200F6000040402FA01F121430160F4E7044AD36813F00103FBD13421D1601361704700BF0F
:200F8000002002400A4B1A6842F001021A601A6891070AD5074B1A69120641BF064A5A6079
:200FA00002F188325A60FFF7E1BF00BFEFE700BF00100240002002402301674508B5FFF7A9
:200FC000D5FF074B1A6942F002021A6158611A6942F040021A61BDE80840FFF7C7BF00BF64
:200FE0000020024070B50C461546FFF7BFFF094E2D1A0444844205EB000200D170BD3369D1
:020000040800F2
:2010000043F00103336130F8023B1380FFF7AEFFF0E700BF0020024070B5154CD4F8903060
:20102000002B23DB002000F05BFCF8B1D4F890600020402E354628BF4025D4F88C102A468E
:2010400000F05AFCD4F88C302B44C4F88C30D4F890305B1BC4F8903043B994F894300BB155
:201060003F2E03D84FF0FF33C4F8903070BD00BF0007002007B5094B094A0A491B68126875
:2010800009680948CDE900212021084AFFF7CEFA03B05DF804EB00F0F1BB00BFE8F7FF1F17
:2010A000ECF7FF1FF0F7FF1FE0060020601E000800F0F4BBF0B50546964C87B008B34FF0FC
:2010C000FF33002008222146C4F89030C4F8880000F00CFC94F90030002B02DBE388002B1A
:2010E00049D194F900302178002B46DBE388802B40F2BD80802219468748FFF771FE002555
:2011000050E0D4F88830002B09DA00F0FBFB2A462946284607B0BDE8F04000F0E7BB94F92F
:201120000030002B1DDB00F0D5FBD4F8881006467F2914D8C1F180028242A8BF0246083178
:201140000020214400F0D2FBD4F88800E38806449E42C4F888600EDBC4F88830C1E72A464B
:20116000EDE70246014600F0C1FB4FF0FF33C4F89030C4F8883007B0F0BD802940F08780BB
:201180006378062B40F08A806288150A012DD2B229D1002A68D161490A786148C4F88820B8
:2011A000FFF709FC94F90030002B80F2AA80E288D4F88830934201DDC4F88820002D00F08E
:2011C000A280574BC4F88C30D4F888309342C4F89030ACBF0023012384F8943007B0BDE8B0
:2011E000F040FFF719BF062D08D1002A3CD100F065FB05460028D5D04A49CDE7022D0ED1F1
:2012000092BB00F061FB40B147498A784448C4F88820FFF7D0FB0125C4E74449F5E7032D97
:2012200022D1032A20D8424B53F822504AB94FF4417323812B88638102235B00C4F8883023
:20124000E9E72846FFF7D6FB00F281104000208138486A1EC5F10205AB1812F8011F00294A
:20126000EBD020F8021BF7E72946334845E771B96378052B05D1A07800F07F0000F04EFBBF
:20128000C9E7092B0AD100F0E5F805468AE701F07F03212B02D100F089F8F6E7E3796278F0
:2012A0000493A379254803936379029323790193E3780093A378FFF793FD94F90030002B60
:2012C0000CDB1F48FFF78CFD0025154E1D4FD4F888309D4206DB1C48FFF782FD1B48FFF7D7
:2012E0007FFD0CE7384616F8011BFFF779FD0135EDE70023C4E9233384F89430FFF78CFE7B
:2013000004E0002DF5D1002000F0FCFA4FF0FF332FE700BF000700206F1E00084E1C00087C
:2013200008070020441C0008BC1B0008001C0008AC1B00080A070020881E0008A41E00089B
:20134000CE1E0008D01E0008D61E0008421E0008FFF762BE37B50E480E4C437B8168052BB6
:2013600028BF0523E35C047B827B64B1012C0CD009480A4D022C18BF284600900848FFF794
:201380002FFD03B030BD0748F7E70748F5E700BF00070020EB1E0008DC1E00086D1E00089D
:2013A000E01E0008DE1E0008D81E000838B5204C6178A1F12003032B35D8DFE803F0021F28
:2013C0001D301C4D1C48FFF70BFDFFF7C3FFA3682A689A4209D042F21072934205D1174B28
:2013E0005B6898471648FFF7FBFC164BA0689A889B792860AA80AB71012018E01248FFF72A
:020000040800F2
:20140000EFFC0C4B0F4A186899889B79A06093719180FFF79FFF0723C4F88830ECE70B480F
:20142000FFF7DEFCE8E70A48FFF7DAFC002038BD0007002018000020F21E0008A41B00089C
:20144000041F000808070020181F00082A1F0008311F000810B500F037FA003818BF012034
:201460000B4B002298720321812000F051FA0221084C0846226800F04BFA02218320226816
:2014800000F046FA044B5B689847012010BD00BF0400002014000020A41B00080020704788
:2014A000024AD36923F40003D3617047001002400C4B13F8103093B10B4A030152F8202084
:2014C00003F18043D10503F5C04304D4D86880B2C0F3090070475206F8D45868F7E74FF0C6
:2014E000FF30704798070020005C0040024B03EB40035878704700BF980700202DE9F041E1
:20150000850005F1804505F5B84594462A68040104F1804412F4807793B204F5C04434D027
:20152000560683EA13224CBFA4682468520603D500261F4A02F81060C4F34E02960006F14D
:2015400080462CF0010E4FEA5C0406F5C0468E4471451FD11CF0010F07D02244920002F1AA
:20156000804202F5C04212680A70C7B1104A23F0F00312F810205B055B0D0AB943F40043A5
:2015800043F0C0032B60BDE8F081094AA46802F81070D1E756F8048B21F8028BD8E723F4CA
:2015A0000F639B049B0C83F4304383F08003E9E7980700202DE9F041850005F1804505F583
:2015C000B8452E68040104F1804416F4807CB3B204F5C04438D076044BBFA6682668E260E8
:2015E000626083EA1324640604D50027214C04EB40046770C6F34E06B70007F1804722F00F
:20160000010E540807F5C0478E44714524D1D20707D5A2199200097802F1804202F5C042AE
:201620001160BCF1000F1CD0124A23F0F00302EB40005B0542785B0D43F440430AB943F0D0
:2016400080032B60BDE8F08126686260094C04EB400484F801C0CDE731F8028B47F8048B19
:20166000D3E723F0C0035B055B0D83F4004383F0B003E6E798070020800000F1804000F580
:20168000B840036823F0C0035B055B0D83F4004383F0900303607047F0B54FFA80FC00F015
:2016A0007F00860006F1804606F5B8463468050105F18045042905F5C045A4B200D100DEE1
:2016C000174BBCF1000F5B5C164940EA43239BB200DB98B90F8A4FF0010E2F6017440F826B
:2016E00000276F6004F0700787F020073B43BCF1000F01EB400787F801E00EDB0F8A04F4A4
:20170000E044AF6017444FF40442EA60002284F440540F82234301F810203360F0BD00BF1B
:20172000601C000898070020014B9874704700BF9807002010B50B4A0B4CD3690A2043F4CB
:201740000003D361236C23F002032364FEF7BAFF236C0A2023F001032364FEF7B3FF002355
:20176000636410BD00100240005C004000207047F8B53A4F7C6CE343250403F4FE437B648C
:201780001BD504F00F05AB0003F1804314F0100F334E03F5B84343D018681A6822F0F0023F
:2017A0005205520D42F080021A60012306F815301DB9C0F3C020FFF77DFC600402D529485A
:2017C000FFF70EFBA10402D52748FFF709FBE20402D52648FFF704FB630520D52448FFF746
:2017E000FFFA244B1B6898471D4B102218460021FFF7C8F84FF0FF311F4AC2F88810C2F86C
:020000040800F2
:2018000090100021402281740282084600F080F88022124BDA645A6C22F480625A64F8BD08
:201820001A6822F0F0025205520D42F400421A60012206EB45035A70002DBED1FFF788FD1D
:20184000B37C002BB9D00C4AD2F89020013202BF43F08003FB64B574AFE700BF005C0040B2
:2018600098070020491F0008531F00085A1F0008621F0008A41B00080007002008B5054BBA
:201880001B689847BDE80840122200210248FFF749BB00BF641C00080008014010B50422E5
:2018A00000210448FFF73EFBBDE81040024B5B68184700BF00080140641C0008014BDB6809
:2018C000184700BF641C0008014B1B69184700BF641C0008014BDB69184700BF641C0008B6
:2018E000014B1B6A184700BF641C0008014B5B6A184700BF641C0008014B9B6A184700BF4B
:20190000641C0008014BDB6A184700BF641C0008014B9B69184700BF641C0008014B5B6902
:20192000184700BF641C0008014B9B68184700BF641C0008000000007819000894190008BE
:2019400000000001681900088019000800000001581900088019000802010900040003002E
:20196000060001000000000002010901040003010600010100000001020109000000000036
:201980000A010B000C0100000E010A0010010100000000000A010B000E010A0000000000CA
:2019A000020100002110422063308440A550C660E770088129914AA16BB18CC1ADD1CEE104
:2019C000EFF13112100273325222B5529442F772D662399318837BB35AA3BDD39CC3FFF3C8
:2019E000DEE36224433420040114E664C774A44485546AA54BB528850995EEE5CFF5ACC548
:201A00008DD55336722611163006D776F6669556B4465BB77AA719973887DFF7FEE79DD787
:201A2000BCC7C448E5588668A7784008611802282338CCC9EDD98EE9AFF9488969990AA987
:201A40002BB9F55AD44AB77A966A711A500A333A122AFDDBDCCBBFFB9EEB799B588B3BBBC7
:201A60001AABA66C877CE44CC55C222C033C600C411CAEED8FFDECCDCDDD2AAD0BBD688DC7
:201A8000499D977EB66ED55EF44E133E322E511E700E9FFFBEEFDDDFFCCF1BBF3AAF599F87
:201AA000788F8891A981CAB1EBA10CD12DC14EF16FE18010A100C230E320045025404670E6
:201AC0006760B9839893FBA3DAB33DC31CD37FE35EF3B1029012F322D232354214527762E7
:201AE0005672EAB5CBA5A89589856EF54FE52CD50DC5E234C324A014810466744764245427
:201B00000544DBA7FAB79987B8975FE77EF71DC73CD7D326F2369106B016576676761546A6
:201B200034564CD96DC90EF92FE9C899E9898AB9ABA94458654806782768C018E108823866
:201B4000A3287DCB5CDB3FEB1EFBF98BD89BBBAB9ABB754A545A376A167AF10AD01AB32AE6
:201B6000923A2EFD0FED6CDD4DCDAABD8BADE89DC98D267C076C645C454CA23C832CE01CA6
:201B8000C10C1FEF3EFF5DCF7CDF9BAFBABFD98FF89F176E367E554E745E932EB23ED10EA6
:201BA000F01E0000390A0008210A0008441E0008471E0008531E0008E006002009024300F5
:201BC00002010080FA090400000102020100052400100104240202052406000105240103B2
:201BE000010705810340001009040100020A00000007050202000200070583020002000045
:020000040800F2
:201C00000902430002010080FA090400000102020100052400100104240202052406000150
:201C20000524010301070581034000FF09040100020A0000000705020240000007058302AC
:201C4000400000000A06000202000040010012010002020000400912694D000101020301BF
:201C60000102000335170008A1140008711700089D1400086D170008291700089916000879
:201C8000B1140008ED140008FD140008B5150008791600083031323334353637383941425C
:201CA00043444546003031323334353637383961626364656600526573657474696E672ECD
:201CC0002E2E0A0049525100457863657074696F6E005468726561640048616E646C6572ED
:201CE00000556E6578706563746564202573202325752061742050433D25303878202825E3
:201D000073293A0A002072303A20202530387820202072313A20202530387820202072321C
:201D20003A20202530387820202072333A2020253038780A002072343A2020253038782031
:201D4000202072353A20202530387820202072363A20202530387820202072373A202025EE
:201D60003038780A002072383A20202530387820202072393A2020253038782020207231A3
:201D8000303A20253038782020207231313A20253038780A00207231323A202530387820A3
:201DA000202073703A2020253038782020206C723A20202530387820202070633A202025F2
:201DC0003038780A00206D73703A20253038782020207073703A20253038782020207073F5
:201DE000723A20253038780A004641494C004F4B000A2A2A204772656173657765617A6C5A
:201E0000652055706461746520426F6F746C6F61646572207625752E25750A005570646123
:201E200074653A2025752062797465730A0046696E616C204352433A2025303478202825DA
:201E400073290A000904004B65697220467261736572004772656173657765617A6C6500E2
:201E600047572530385825303858253038580043746C204F555420746F6F206C6F6E673A5E
:201E80002025753E25750A005B556E6B6E6F776E2064657363726970746F722025752C25F1
:201EA000755D0A00282530327820253032782025303278202530327820253032782025302E
:201EC00032782025303278202530327829005B002530327820005D00312E35003200310023
:201EE00025752C2575256325730A006E6F656D733F005345545F4C494E455F434F44494EB8
:201F0000473A2000436F6D6D73204C696E6520436C65617265640A004745545F4C494E4538
:201F20005F434F44494E473A2000425245414B0A005B436C6173732D737065636966696301
:201F40003A20253032785D0A005B504D414F56525D0A005B4552525D0A005B574B55505D80
:201F60000A005B52455345545D0A00000000001600000000010000000000000040000000BB
:201F80008025000000000800FFFFFFFFFFFFFFFFFFFFFFFFFFFFFFFFFFFFFFFFFFFFFFFFAC
:201FA000FFFFFFFFFFFFFFFFFFFFFFFFFFFFFFFFFFFFFFFFFFFFFFFFFFFFFFFFFFFFFFFF41
:201FC000FFFFFFFFFFFFFFFFFFFFFFFFFFFFFFFFFFFFFFFFFFFFFFFFFFFFFFFFFFFFFFFF21
:201FE000FFFFFFFFFFFFFFFFFFFFFFFFFFFFFFFFFFFFFFFFFFFFFFFFFFFFFFFFFFFFFFFF01
:020000040800F2
:202000000806002095280008ED270008ED270008ED270008ED270008ED270008ED27000825
:20202000ED270008ED270008ED270008ED270008ED270008ED270008ED270008ED270008C0
:202040005121000851210008512100085121000851210008512100085121000851210008B0
:20206000512100085121000851210008792800085121000851210008512100085121000861
:20208000512100085121000851210008512100085121000851210008512100085121000870
:2020A00051210008A12500085121000851210008512100085121000819280008512100082D
:2020C000512100085121000851210008512100085121000851210008512100085121000830
:2020E000512100085121000851210008512100085121000851210008512100085121000810
:202100005121000851210008512100085121000851210008512100085121000851210008EF
:202120005121000851210008512100085121000851210008512100085121000851210008CF
:20214000512100085121000851210008512100082DE9F04F684600F081B92DE9F007B1E8C4
:20216000F807A0E8F807203AF9D1BDE8F00770472DE9F007CDB24FF001346C4323462546DF
:2021800026462746A046A146A246A0E8F807203AFBD1BDE8F007704703688B4238BF1A70F8
:2021A00003680133036070472DE9F04F8046174687B01D464B1E02900093C118BA461AF8DB
:2021C000012B52B9029B8B4200F2FA801A700298A0EB080007B0BDE8F08F252A04D002A893
:2021E000FFF7DAFF5746E9E7002634461CE0A2F16303152B26D8DFE803F072562525253EA1
:20220000562525252525491125255B2558252511392A21D9582A15D144F4807444F010049F
:2022200036E055F8046BBA46574617F8012B782A08D8622ADBD8302A0BD0E9D8232A05D01B
:202240002A2AEED002A8FFF7A7FFB7E744F48064E9E744F40064E6E7A2F130063A4612F8E0
:20226000013BA3F130000928DDD80A2000FB06361746303EF2E79AF80130682B06BF44F420
:2022800080540AF1020744F40054CCE744F00804E30455F8049B04F4007224D55FFA89F9D6
:2022A00024F4007432E044F4007444F00A04EFE755F8044B2644A6EB040A14F8012B52B9D4
:2022C000BAF1000F7FF77AAF202202A8FFF764FF0AF1FF3AF4E702A8FFF75EFFEBE755F835
:2022E000042BD2B2AEE7A00437D59AB30FFA89F9B9F1000FD4DA230505D52D2202A8FFF7B6
:202300004BFF24F40074013EC9F1000960050FD504F01F0ABAF1080F02D0BAF1100F07D149
:20232000302202A8FFF738FFBAF1100F18D0013E0DF10C0AB9F1000F18D130230DF10D0B64
:202340008DF80C3014F4006F14BF30222022ABEB0A0327E01FFA89F9A2E7002AA0D0C7E7C8
:20236000782202A8FFF718FF023EE1E7D346174A14F4807F164808BF104604F01F02B9FB3F
:20238000F2FC02FB1C9E10F80EE00BF801EBCE467245E146F3D9D5E702A80193FFF7FCFE0B
:2023A000019B013EB342F7DBA30503D52D2202A8FFF7F2FED3453FF401AF1BF8012DF6E703
:2023C00088459CBF009B08F8032000E7B52E0008A42E0008EFF3088181F30988022181F364
:2023E0001488BFF36F8F104B83F308880F4B104A9A605A6942F404725A615A6A42F4E0225C
:020000040800F2
:202400005A624FF07F42DA614FF47F021A62BFF34F8FBFF36F8F6FF07F42A3F54F635A6021
:2024200001221A60704700BF0802002000ED00E00020000808B572B6054800F029FCBFF371
:202440004F8FBFF36F8F034B034ADA60FEE700BFC62E000800ED00E00400FA05F7B50446B3
:20246000EFF30382006AD2B2410704F1240341D5EFF309851E4605F120070F2A40D82249E0
:20248000DFF8A8C010F0080F204808BF6046AB6900901F4800F0FCFBEB681E480093D5E915
:2024A0000123296800F0F4FBE368216800931A48D4E9012300F0ECFBE3692169009317483F
:2024C000D4E9052300F0E4FB236A296913F0040FAB6918BF3A46009308BF32466B691048AA
:2024E00000F0D6FB3A463146EB690E4800F0D0FBFFF7A0FFEFF309871D4604F14406BCE773
:202500000949103ABCE700BFD82E0008E22E0008F12E0008152F0008452F0008752F0008FC
:20252000A52F0008D52F0008D42E0008E92E0008064B074A1B68926803F07F4010438342A1
:2025400038BF00F17F40C043704700BF0806002010E000E00C22114BB0F5803F1A600FDA0C
:202560000D284FF00702B8BF0D209A620C380122D8620A4B5A6100221A610D221A60704790
:2025800041F61F429A624FF4617290FBF2F04FF6FF723238904228BF1046E8E7002C0140B9
:2025A0000022F8B501270B4B0B4E1A61346804B9F8BD2568FFF7BCFF281A0C2803DDBDE8B3
:2025C000F840FFF7C7BFE368E7603360D4E901309847EBE7002C01401C060020F8B532F005
:2025E0001F0506460F4614460CD083070AD12A46FFF7BEFD04F01F0472191444A24203D1A8
:202600003046F8BD3246F8E702F8017BF6E7F8B532F01F0706460D46144610D040EA0103E9
:202620009B070CD13A46FFF798FD3D44F31904F01F04013B2C44A54203D13046F8BD334661
:20264000F7E715F8012B03F8012FF4E7034610B502449A4201D1002005E013F8010B11F836
:20266000014B001BF5D010BD044B186880EA403080EA504080EA40101860704704000020B1
:20268000012208B5064B07481A7000F001FB4FF48052054B1A614FF40052C3F8102408BD1B
:2026A00020060020F92F0008000C014010B1024800F0EEBAFFF7E4BF0530000810B50446CF
:2026C000124800F0E5FA002323601023A36040F22473636040F201432360A368102B05D154
:2026E0002368012B02D10A4800F0D2FAA368102B09D140F201432068C31A58425841BDE86F
:202700001040FFF7D3BF0020F9E700BF093000081B30000810B504460B4800F0B9FA41F652
:202720001F430122A36241F28733E362E2600022626005222260E06ABDE81040C31A584258
:202740005841FFF7B3BF00BF293000082DE9F0410D4607461146204800F09AFA4FF00008E7
:2027600001234FF480621D4E122173602846C6F8088077613561F260FFF730FF44F2D303FA
:20278000174CC4F80480B3606368002BFCD06368012B04DD61681348013900F079FA4FF4E5
:2027A000806229463846FFF751FF10B10E4800F06FFA6368012B0CD14FF4806229463846AE
:2027C000FFF744FFB0FA80F04009BDE8F041FFF76DBF0020F9E700BF3B30000800000240F1
:2027E000200600204C3000086830000808B5EFF3038172B60648C9B200F04AFA4FF4805212
:020000040800F2
:20280000044B1A614FF40052C3F81024FEE700BF74300008000C01400022124B1A61124A77
:2028200013784BB14FF08042104BC3F88020BFF34F8FBFF36F8F7047137A0D49002B14BF82
:202840004FF480504FF08050086114BF4FF400504FF0005083F00103C1F8100405481372E2
:2028600000F016BA000800402006002000E100E0000C0140603200080122044B5A60002214
:202880009A60034A536801335360704700000240200600202DE9F04FB948BA4985B08842B8
:2028A00003D0B94A121AFFF7B2FEB848B84FB94C00213A1AFFF792FE00F016FAE369B64D1A
:2028C00043F0C053E36100F0F1F9B44800F0E0F9B34800F0DDF9B34800F0DAF916220C21EB
:2028E000B14800F065FA16220D21B04800F060FAAF4BB048B04E19885A8804331B88008813
:202900002D88368880B2ADB2B6B200909BB292B289B2CDE90156A94800F0BAF9A84BA9486A
:20292000B3F800901FFA89F9494600F0B1F9B9F1400F00F0088108D8B9F1100F0AD0B9F1F9
:20294000200F00F0F880A048FEE0B9F1800FFAD19E48F9E09E4800F09BF903264FF001087C
:2029600006259C4800F094F99B4B9C48D3F800A0CAF30B0100F08CF999484FEA1A4100F0F3
:2029800087F9BAF1000F02D0964800F081F9E369012143F400139448E361FFF78FFEB8F1DF
:2029A000020F07D1E369414643F480038F48E361FFF784FE4FF0030B40F64D3AA3690121D6
:2029C00043F48053A3618A4800F062F9894BC3F804B0C3F800A05868A0EB0B0250425041B3
:2029E000FFF764FEB8F1020F13D1E369414643F48043E3617E4800F04BF97F4BC3F804B09D
:202A0000C3F800A05868A0EB0B0358425841FFF74DFE01217948FFF77DFE02214FF0804018
:202A2000FFF778FE03217648FFF774FE042E03D131467448FFF76EFE01224021724B5A604A
:202A4000724B83F80B134FF40061C3F88011704C196020464E49FFF779FE601C02224C495C
:202A6000FFF774FE204603226A49FFF76FFE0422601C6849FFF76AFE4946674800F008F96D
:202A800000F0C6F9654B4B4404EB8328404600F0DBF94FF48062FF213D48FFF79FFD4FF4C5
:202AA000806240463A49FFF7D1FD0446002852D1FFF7DAFD38510434B4F5806FF8D142465B
:202AC0002146334800F0D4F9224640463049FFF7BDFD00283FD1524800F0DAF8042E3DD16C
:202AE000504800F0D5F84022484B83F81E234FF08042C3F880214A481A6000F0C9F8294647
:202B0000494800F0C5F8494905F500250E46204CAD0222460F6895422DD8224637609542C6
:202B2000F7D952F8047BFFF79FFD8742F7D0FFF7A7FD72B6FEE73E4800F0AAF803264FF0B3
:202B400001080A250DE73B4800F0A2F804264FF00208142505E7FFF793FDBFE7364B1B7864
:202B6000002BCCD14FF080520F4B1A614FF00052C3F81024C3E7FFF777FD42F8040BCAE719
:202B800004000020643200080800002008060020B406002000100240F0F7FF1F9030000824
:202BA000A4300008C9300008000C014000100140E8F7FF1FEEF7FF1FF2F7FF1FF330000868
:202BC000E0F7FF1F1B310008953100087A3100082F310008A4310008002004E0A731000802
:202BE000BB310008CF3100080054004000580040013200080030014000380040002C01401C
:020000040800F2
:202C000000040040000800400000024000E100E000200008B506002013320008FFFF3F0098
:202C2000053000082A3200083E32000804000020473100085F3100082006002070B502468C
:202C40000B46EFF3108404F0010472B60D2580210D48FFF7A9FA0C490C4A11F8013B13B90F
:202C600004B962B670BD0A2B07D00D2BF5D01668360607D55360F0E700BF16683606FBD5E0
:202C80005560F4E700BFF2E729060020003801400FB407B504A951F8040B0191FFF7CEFF6B
:202CA00003B05DF804EB04B07047000010B50B4A0B4C9369204643F480439361092211466F
:202CC00000F076F818220A21204600F071F81822044B9A6042F20C02DA6010BD0010024054
:202CE000000801400038014008B5FFF773FB2B4B2B4A1B889BB2102B136003D0202B45D035
:202D0000142300E0062353601222264B1A60A3F580531A6842F480321A601A68910337D530
:202D2000214A5A601A6842F080721A601A68920130D55A6842F002025A605A6802F00C02C0
:202D4000082A29D11A6822F001021A600722DA6140F61D029A6101225A614FF08062134B25
:202D60005A604FF0443302F1705202F5843253601360C2F80434C2F80034C2F80438C2F8CB
:202D80000038BFF34F8FBFF36F8F08BD0A23BAE700BFC2E700BFC9E700BFCEE7E0F7FF1FE8
:202DA000AC0600200020024000C41D0000000140130914BF01234FF48033072903FA01F393
:202DC00030B503614FF00F0402F00F020AD9083945688B009C4025EA040402FA03F32343AE
:202DE000436030BD036889008C4023EA040402FA01F121430160F4E7044AD36813F0010350
:202E0000FBD13421D1601361704700BF002002400A4B1A6842F001021A601A6891070AD595
:202E2000074B1A69120641BF064A5A6002F188325A60FFF7E1BF00BFEFE700BF00100240F8
:202E4000002002402301674508B5FFF7D5FF074B1A6942F002021A6158611A6942F0400283
:202E60001A61BDE80840FFF7C7BF00BF0020024070B50C461546FFF7BFFF094E2D1A0444E1
:202E8000844205EB000200D170BD336943F00103336130F8023B1380FFF7AEFFF0E700BFE4
:202EA0000020024030313233343536373839414243444546003031323334353637383961A0
:202EC000626364656600526573657474696E672E2E2E0A0049525100457863657074696F88
:202EE0006E005468726561640048616E646C657200556E657870656374656420257320233E
:202F000025752061742050433D2530387820282573293A0A002072303A202025303878207F
:202F2000202072313A20202530387820202072323A20202530387820202072333A20202508
:202F40003038780A002072343A20202530387820202072353A2020253038782020207236B4
:202F60003A20202530387820202072373A2020253038780A002072383A20202530387820D7
:202F8000202072393A2020253038782020207231303A20253038782020207231313A202582
:202FA0003038780A00207231323A202530387820202073703A2020253038782020206C72D3
:202FC0003A20202530387820202070633A2020253038780A00206D73703A202530387820C7
:202FE00020207073703A20253038782020207073723A20253038780A002A2A4641494C450C
:020000040800F2
:20300000442A2A0A004F4B0A0054657374696E672049324325642E2E2E20005B46616B65A9
:2030200020436869703F5D200054657374696E672054494D25642E2E2E2000444D412054CF
:20304000657374202325752E2E2E20005B53707572696F7573204952513A2046616B6520DB
:20306000436869703F5D20005B42616420446174615D20002A2A4641494C45442A2A205BCF
:20308000457863657074696F6E202325755D0A000A2A2A20426C696E6B7920546573742076
:2030A0002A2A0A002A2A204B65697220467261736572203C6B6569722E78656E40676D613B
:2030C000696C2E636F6D3E0A002A2A2068747470733A2F2F6769746875622E636F6D2F6B9D
:2030E000656972662F4772656173657765617A6C650A0053657269616C203D202530347834
:203100003A253034783A253034783A253034783A253034783A253034780A00466C61736890
:203120002053697A65203D2025756B4220280053544D3332463130337834204C6F772D4426
:20314000656E736974790053544D3332463130337836204C6F772D44656E73697479005340
:20316000544D3332463130337838204D656469756D2D44656E736974790053544D33324692
:203180003130337842204D656469756D2D44656E7369747900556E6B6E6F776E2044657624
:2031A00069636500290A00446576696365204944203D203078253034780A00526576697375
:2031C000696F6E20203D203078253034780A002A2A5741524E494E472A2A3A2044657669B9
:2031E00063652072657475726E65642076616C6964204944434F4445212046616B653F0A85
:203200000054657374696E672053504925642E2E2E200054657374696E672025756B42202C
:20322000466C6173682E2E2E2000456E61626C652054494D34204952512E2E2E2000546502
:203240007374696E672025756B42205352414D2028656E646C657373206C6F6F70292E2EFA
:203260002E0000003C26A287FFFFFFFFFFFFFFFFFFFFFFFFFFFFFFFFFFFFFFFFFFFFFFFFAD
:20328000FFFFFFFFFFFFFFFFFFFFFFFFFFFFFFFFFFFFFFFFFFFFFFFFFFFFFFFFFFFFFFFF4E
:2032A000FFFFFFFFFFFFFFFFFFFFFFFFFFFFFFFFFFFFFFFFFFFFFFFFFFFFFFFFFFFFFFFF2E
:2032C000FFFFFFFFFFFFFFFFFFFFFFFFFFFFFFFFFFFFFFFFFFFFFFFFFFFFFFFFFFFFFFFF0E
:2032E000FFFFFFFFFFFFFFFFFFFFFFFFFFFFFFFFFFFFFFFFFFFFFFFFFFFFFFFFFFFFFFFFEE
:020000040800F2
:00000001FF
